:020000040000FA
:020000001729BE
:08000800FD00030EFC00831251
:100010008C1C68288C10B6182928B61D68280A0878
:10002000FE008A014808C6070318C70A4908C7071F
:10003000470C7F397E20211C2128C1000310410C70
:10004000403EFF2041089300420895007E088A0048
:1000500068284108930042089500AF08031D47280F
:100060002D082E0403196628BD080319BE03BD031D
:100070003D083E04031D66282D08BD002E08BE0065
:10008000A725F101F2018625B61BE12B672809217E
:1000900003195728F20A0319F10A72087104031DA3
:1000A0006628A725F101F2014508F30062282D0812
:1000B000BD002E08BE002F08BF00A725F101F201E8
:1000C0004408F3008625B61BE12B6728A125FF20F5
:1000D0000C1C79280C10B90B792838140530B9009C
:1000E0000A30BA073C303A02031D7928B814BA0125
:1000F000BB0A7C0E8300FD0E7D0E09008207803452
:1001000086348C34933499349F34A534AB34B13471
:10011000B634BC34C134C734CC34D134D534DA34F9
:10012000DE34E234E634EA34ED34F034F334F534DA
:10013000F834FA34FB34FD34FE34FE34FF34FF343B
:10014000FF34FE34FE34FD34FB34FA34F834F53435
:10015000F334F034ED34EA34E634E234DE34DA34C5
:10016000D534D134CC34C734C134BC34B634B134D2
:10017000AB34A5349F34993493348C348634803432
:100180007A3474346D34673461345B3455344F34AD
:100190004A3444343F34393434342F342B34263405
:1001A00022341E341A341634133410340D340B3404
:1001B0000834063405340334023402340134013483
:1001C00001340234023403340534063408340B3469
:1001D0000D341034133416341A341E3422342634B9
:1001E0002B342F34343439343F3444344A344F348C
:1001F00055345B34613467346D3474347A34C100FF
:10020000410E30390C38C200C10CC10C3F30C10561
:100210000800BD0B0E293E083F04080003113D0FE6
:100220000800BE0B3E0F0800BF0B0800080083014A
:100230008B018A0185018701073099006400D23063
:1002400083168100910170308F00073085001030D7
:100250008700811783120711203084008001840AEF
:100260007F300402031D2E29203084001030F0005E
:10027000003083169B001C141A088000840A9B0A15
:10028000F00B3B298312290883169000831217264E
:100290002D26B6010E30900080308F008E010C109C
:1002A00010141E30BC00643044260C185B29BC0BB3
:1002B00053290330E22B10100C108E018F0196246D
:1002C0000230BC00C308031DBC0A0714C830442612
:1002D0000710C8304426BC0B652905197329201C5A
:1002E000AA29A018AA290710FA2303188729051993
:1002F0007329AD22FA30BC00051973290230442657
:10030000BC0B7C290714051D82290710AA29AD22E0
:10031000FE232124563A03195F2B563A443A031917
:10032000A12B443A553A0319B92B553A543A0319BB
:10033000AA29543A523A0319772B523A573A0319D9
:10034000822B573A433A0319662B433A403A031932
:10035000002873293611A808031D36152112AB0891
:10036000031D211610103810B8100530B900BA015D
:10037000BB018F018E010C1083160C1483120B1716
:100380008B171014A2080319D02963000000381C31
:10039000C529F5233810B81CC529B810A20BC529EA
:1003A0002018EA29071487146430442687156D2223
:1003B000201FDD29A1188711B611201B6B24A0195D
:1003C0003D24A01B4D242019D124B81CDD29B810D0
:1003D0002623DD29A018282AB4012308B500240803
:1003E0003406031D102A0714871464304426871529
:1003F0006D22201FFE29A1188711B611172200387F
:10040000031D0B2A201B6B24A0193D24A01B4D2487
:100410002019D124FE297B22871187100710EF298C
:1004200063000000172200380319102AEF29381C36
:1004300000343810B50B00342308B500B40A340872
:1004400025060319B401B81C0134B8102623013461
:10045000B4010830A5000310340D103E83169B0034
:100460001C141A088312A300A308031D392AB4011F
:100470002B2A2308B50083169B0A1C141A08831222
:10048000CF004F1C662AFC30CF05200803394F04EB
:10049000A000071487146430442687156D22201F9E
:1004A000542AA1188711B61117220038031D612A9A
:1004B000201B6B24A0193D24A01B4D242019D124FE
:1004C000542A7B228711871007102B2A6300000013
:1004D000172200380319662A2B2A201AA52AA01AE7
:1004E000872A201BBB2AA01BB32AA019BE2A2019C9
:1004F000C02A2016A52A201AAD2AA01A9A2A201B43
:10050000AD2AA01BAD2AA019AD2A2019AD2A2D08AD
:10051000BD002E08BE002F08BF00F101F201440803
:10052000F3008B138B1B912A86258B17B61BE12BAF
:10053000B614C72A83168C1083121211B6108B13AF
:100540008B1B9F2AA7258B1708002608C8002708A1
:10055000C900C601C701B615C72A83168C108312BD
:100560001211B6110800CE01C8010330C900C6013E
:10057000C701B615C72AF822CA01A52ACA01A52AA9
:100580002F25D708031DA52A20112016A52A1830CB
:100590009200910183163F30920083121F30930026
:1005A0003C3095008C1083168C1483120B178B171C
:1005B000121508004B30840040304A0783169B0018
:1005C0001C141A088000840A9B0A1C141A08800054
:1005D000840A9B0A1C141A08800083120330CA077D
:1005E0004A08303A0319CA01CB080319DA2A08006D
:1005F0002119092BA0308400203083169B001C1485
:100600009B0A1A088000840A0038031DFF2A8312FF
:100610000800A03084004D308000840A4F308000F4
:10062000840A201C172B2408213E8000840A2030D5
:100630008000840A80010800A0304A078400000876
:10064000CA0A0038031D0800CA011C2B361D080009
:10065000A80B0800211A352B8B138B1B2C2B900118
:1006600092018711871007106300AB080319492B0B
:10067000871187100710B611B610910163000000B2
:10068000381C3E2BF5233810B81C3E2BB810AB0B92
:100690003E2B900107148714643044268715A52249
:1006A000FA304426FA304426AD228711871007100D
:1006B000FA304426FA30442696304426492B430823
:1006C000033910382124203021247329FE232124CA
:1006D000B700B71B732937081F39831690008312A0
:1006E00007140000732B0710071E702B662BBC012C
:1006F0003C0883169B001C141A0883122124BC0F8B
:10070000782B7329FE2383169B0083122124FE235A
:10071000BC002124FE2383169A001C158B138B1B0F
:100720008E2B55309D00AA309D009C148B179C1871
:10073000972B1C119B0A831223302124BC0B8A2B7C
:100740007329FE23BC002124FE2364252124FE23DB
:10075000F1002124FE23F20021246B25B61BE12B9E
:1007600074082124B613AD25B61BE12BBC0BB02BAE
:100770007329FE23F4002124FE2364252124FE2373
:10078000F1002124FE23F2002124C0017408B700E7
:10079000A0308400FE238000C007840AB70BCA2B58
:1007A00040082124FE232124473C031D7329A03047
:1007B00084000714B9250710B61BE12B2330212430
:1007C000732902308B138B1BE22B8312B70037087F
:1007D000BC00F523C8304426BC0BE92B0330BC0019
:1007E000FF304426BC0BF02BE72B07141E304426A9
:1007F000071008000310071A03140800071EFE2B39
:100800000830B100B0010F30B200B20B052C00006F
:10081000071EFE2B0B2C00002030B200B20B0E2C5A
:100820000310B00C071EB017B10B0C2C2030B20017
:10083000B20B182C03101C2C0000071A03143008EC
:100840000800B0000830B10007152130B200B20B2B
:10085000272CB00C031C0715031807111F30B2001A
:10086000B20B302C332CB10B292CB00C07114230B9
:10087000B200B20B392C30080800DA228B138B1B24
:100880003E2C4C08C8004D08C9008B170A30B70031
:100890004B084426B70B482C08000A3044264E1853
:1008A0005E2C8B138B1B512C1030C8070318C90A00
:1008B0008B1749081E3A03194E1408008B138B1B23
:1008C0005E2C1030C802031CC9038B174908023A7A
:1008D00003194E1008001C23B00007308A003008AE
:1008E00080278A01B000B0080319902C0310B00CC7
:1008F000B0080319852C031C7F2C8824802C8C24A1
:10090000A1188711B6119324762C93249324080000
:10091000A1188715B615912CA1188715B615932C1B
:100920009324932493242A0844260800C301C40175
:10093000C501F101F201A030F3006B25B61BB62C06
:100940001726B613A830F3006B25B61BAE2CA830C3
:10095000C400A030C5000330C30008001726B6133A
:10096000A030C400C5000230C30008001726B6132B
:10097000AA30F3006B25B61BC42CA830C400AA30E3
:10098000C5000330C30008001726B613A830F300D3
:100990006B25B61B0800A830C400C5000230C30098
:1009A000080056085706031DD72C0630D6005125DF
:1009B0005908DB005808DA00501FE92C0310590CC5
:1009C000B100580CB0003008DA070318DB0A310810
:1009D000DB0707308A0050080F39D227CC005008B7
:1009E0000F39C327CD008A015308D500D01EFC2C37
:1009F000510D7039D500D50E5208D400501E032D6C
:100A000051080739D400540803190B2D0310CD0CDD
:100A1000CC0CD40B062DD5030319122D0310DB0CBF
:100A2000DA0C0B2D8B138B1B122D4C08C8004D08B4
:100A3000C9008B1701304426DA080319DB03DA03F7
:100A40005A085B04031D1A2DA11D08008B138B1B74
:100A5000262DC801C9018B17143044260800D60181
:100A6000D701512551080739D200510D7039D300F3
:100A7000D30E5125D801D00CD80C500CD80C1F39EE
:100A8000D90051083F39D8045125A111501BA11597
:100A9000D701D00CD70C500CD70C51083F39D704D4
:100AA00008008030560783169B001C141A08831216
:100AB000D000D60AD01F080083169B0A1C141A08FF
:100AC0008312D100D60A0800B70044083718450839
:100AD000F30037080800831604267308FE39E22560
:100AE0007618412E7108E2257618412E7208E2250B
:100AF0007618412E8510042673080138E2257618F1
:100B0000412ED2250C267408831208008316042671
:100B10007308FE39E2257618412E7108E225761811
:100B2000412E7208E2257618412E8510042673089E
:100B30000138E2257618412ED22523268312740827
:100B400008008316D2252326740883120800831612
:100B5000D2250C2674088312080083160426730815
:100B60000138E2257618412ED2250C26740883120E
:100B70000800831604267308FE39E2257618412EF4
:100B80007108E2257618412E7208E2257618412E6A
:100B90000008E2257618412E840AF40BC82D0C2695
:100BA00083120800F4010830F000F40D85100000F5
:100BB000000085148312051CDE2D74148316F00BBF
:100BC000D52D0800F5000830F000F50CF50D851066
:100BD000F51BEC2D0510EE2D051400008514F00B0F
:100BE000E62D000085100000051400008514F001BA
:100BF0008316F00A0319022E83120518F82D8316A6
:100C000076100800761408000514062E00008514DE
:100C1000092E00000510080085100E2E000005109A
:100C2000112E00008514142E0000051408008312F4
:100C3000F6010508FC39850083161E2E0514202EAA
:100C4000851483120800851000000510000085142B
:100C5000292E85100000051408008316042685102F
:100C6000312E000005140930F0008514372E0000E5
:100C700085103A2E0000F00B352E04260C26831228
:100C800008008312B6170800F00081010B1106302E
:0C0C900081070B1D492EF00B462E0800BA
:100F0000E03E3F39820700340234043408341034A0
:100F10002034403480341F343F347F34FF34733402
:100F200000346A3429343F343E343C34383430346D
:100F300020342134233427342F34473455340034BB
:100F4000003400344C34563406341134153409342A
:100F5000023414340B34103404341E340D3412347F
:100F6000073405340F3416341B340A340834033480
:100F70000C3418340E3419341D341334AA340034AC
:100F8000D534003400340F398207003439343C340E
:100F90004034443448344C34513456345B34603437
:100FA00066346C34820700348334F234923465340E
:100FB0007B34C33456342C344D34BA347A347E34D2
:02400E00E43399
:104200001000000000000600000002000000100086
:10421000F0000000C80000000000000000000000E6
:1042200001008100010041000100000000000000C9
:10423000000000000000000000000000000000007E
:10424000500045003100470052004C00200054004F
:0842500053005400200000009F
:10428000050012000D000A009B0013000F0024001F
:104290001A001400AE0020001900370027001E008D
:1042A000C0002D002300490034002800C0002D006C
:1042B0002D00370027003200AE0020003700240018
:1042C0001A003C009B0013000000000000000000EA
:1042D00000000000000000000000000000000000DE
:104300008000A2009700DC0080007E000B00090006
:104310000B000900A8001800A4001800A000180055
:10432000080009000B0009000B0009000800090043
:104330000B0001000200010002000100AB001800A8
:10434000A0001800AC001800AB001800AA0018006C
:10435000A90018000700060004000600A7001800C6
:10436000A00018000700060004000600A7001800BF
:0C437000A4001800AB001800A00018000A
:00000001FF
